:02000000502886
:1000060083120313CB01CA01C9018030C800C10C99
:10001600C00C031C17284408C90745080318450FD8
:10002600CA070318CB0A0310C01F1F284408CA07B3
:1000360045080318450FCB07CB0CCA0CC90CC80CD6
:10004600031C0A284B08C3004A08C2004908C1001D
:060056004808C00008008C
:10005C00831285140630CB001330CC00AD30CD00AC
:10006C00CD0B3628CC0B3628CB0B362800000000E5
:10007C0005140630CB001330CC00AD30CD00CD0BC9
:10008C004528CC0B4528CB0B4528000000008510DB
:04009C000510080043
:1000A0000F308316860085018F018312061786198B
:1000B0005B2801308F0006195F2802308F078618F1
:1000C000632804308F070618672808308F07061347
:1000D0009001861686196E28013090000619722844
:1000E00002309007861876280430900706187A2880
:1000F0000830900786129101061686198128013072
:100100009100061985280230910786188928043045
:10011000910706188D280830910706128D018E016F
:100120001108C000C1016430C400C50103204008AB
:100130009200410893001008C000C1010A30C400B9
:10014000C50103201208C00713080318013EC107A8
:100150000F084007C20041080318013EC3004208CF
:100160008D0043088E0000304302031DB928033080
:1001700042020318BE288510051054282E20013095
:100180008C0002300D02C1000030031C013E0E0243
:10019000C20000304202031DCF280C084102031C9C
:1001A000E9280630CB001330CC00AD30CD00CD0BAC
:1001B000D728CC0BD728CB0BD72800000000003065
:1001C0004206031DE52841080C060319E9288C0A9C
:0601D000C128BE28EA2848
:02400E00FA3F77
:00000001FF
